:1000000045C0000058C0000056C0000054C00000A9
:1000100052C0000050C000004EC000004CC00000A4
:100020004AC0000048C0000046C0000044C00000B4
:1000300042C0000040C000003EC000003CC00000C4
:100040003AC0000038C0000036C0000034C00000D4
:1000500032C0000030C000002EC000002CC00000E4
:100060002AC0000028C0000026C0000024C00000F4
:1000700022C0000020C000001EC000001CC0000004
:100080001AC0000018C0000016C0000011241FBED6
:10009000CFEFD0E4DEBFCDBF11E0A0E0B1E0E4E2FD
:1000A000FEE000E00BBF02C007900D92A230B10746
:1000B000D9F7BCD5B5C6A4CFBF92CF92DF92D901F4
:1000C000E6E4F0EF0F921F92D72EC62EB82E242F03
:1000D0001B2E0A2E09952131F9F71F900F90DF9002
:1000E000CF90BF900895BF92CF92DF92D901E6E4FE
:1000F000FEEF0F921F92D72EC62EB82E242F1B2E46
:100100000A2E09952131F9F71F900F90DF90CF90BB
:10011000BF900895CF93DC01280F391FA217B307B2
:1001200049F06BBFFA01C791CD934F5F5F4F6F4F9F
:100130007F4FF4CFCF910895CF93DF93FA01E90178
:10014000C13021E0D20710F0C0E0D1E0AB01BC012A
:1001500044279E01CF01DEDFCE01DF91CF910895CC
:100160002F923F924F925F926F927F928F929F92C7
:10017000AF92BF92CF92DF92EF92FF920F931F93B5
:10018000CF93DF93E901C13021E0D20710F0C0E046
:10019000D1E01E01369427946B017C01CC245A01D6
:1001A000DA012601370120E030E060E070E022153E
:1001B0003305C9F06BBEF201879196914D915D9127
:1001C0008417950709F071E040955095842B952B85
:1001D000019609F061E082E0480E511C611C711C1F
:1001E0002F5F3F4FE4CF772351F1662339F020E0B2
:1001F00030E043E0C701B601F80109952601370157
:10020000812C912C8214930491F0F501219131916C
:100210005F0141E0C301B201F8010995F2E04F0E20
:10022000511C611C711C2FEF821A920AEBCF20E047
:1002300030E045E0C701B601F801099502C0C0E011
:10024000D0E0CE01DF91CF911F910F91FF90EF9001
:10025000DF90CF90BF90AF909F908F907F906F90E6
:100260005F904F903F902F9008957EC00000BFC0D8
:100270000000A3C00000A1C000009FC000009DC0FE
:1002800000009BC0000099C0000097C0000095C00E
:10029000000093C0000091C000008FC000008DC01E
:1002A00000008BC0000089C0000087C0000085C02E
:1002B000000083C0000081C000007FC000007DC03E
:1002C00000007BC0000079C0000077C0000075C04E
:1002D000000073C0000071C000006FC000006DC05E
:1002E00000006BC0000069C0000067C0000065C06E
:1002F000000063C00000BBBEEC2DFD2DB7B6B0FC06
:10030000FDCF27BFE895B7B6B0FCFDCF21E1B7B66A
:10031000B6FCF4CF089509021200010100803209F1
:10032000040000000000000012011001FF0000089E
:10033000C016DC050201010200010E035500530046
:1003400042006100730070001C03770077007700A3
:100350002E00660069007300630068006C002E00C8
:10036000640065000403090411241FBECFEFD0E42C
:10037000DEBFCDBF24B7D0E4CEEF3991303F399105
:1003800009F03FEF30933E0120933D0111E0A0E0E2
:10039000B1E0ECEBF9EE01E00BBF02C007900D926B
:1003A000A630B107D9F721E0A6E0B1E001C01D9267
:1003B000AD33B207E1F78CD134C457CFA82FB92F92
:1003C00080E090E041E050EA609530E009C02D9176
:1003D00082279795879510F084279527305EC8F37C
:1003E0006F5FA8F30895EADF8D939D930895CF93EF
:1003F000CFB7CF93DF93C395499BE9F7499B0BC0D8
:10040000499B09C0499B07C0499B05C0499B03C044
:10041000499B01C089C06F93C0912001DD27C95D50
:10042000DE4F2F9365E5499B03C02F916F91E6CF77
:100430000F931F934F9320E040E15F9309B1067043
:1004400001FB27F93F9350E03BE039C01670406450
:100450002F77012F5F5F1EC0406819B116702F778C
:1004600052501FC0406409B12F770670D1F15F5F11
:1004700000C023C0406219B12F77167091F15F5F01
:1004800000C025C006701027515012F45D5F0000B7
:10049000115027952C3F19B1C8F61670012701504D
:1004A00027952C3FC8F64227499309B106701027BB
:1004B0004F73115027952C3FA8F64695469519B1D4
:1004C000167079F00127015027952C3F98F66B5A4A
:1004D00060F3315009B1B0F600C011E01CBB002739
:1004E00017C03B503195C31BD04011E01CBB0881A5
:1004F000033CF9F00B34E9F020911E011981110F32
:100500001213EDCF093651F10D3211F0013E39F7DA
:10051000009325013F915F914F911F910F912F9172
:100520006F91CCB3C0FD67CFDF91CF91CFBFCF919B
:10053000189520912501222369F31091230111239D
:1005400039F534303AF13093230120931F01109193
:1005500020013BE0311B309320011CC0009123019E
:100560000130B4F40AE53091010134FD14C0009368
:100570000101C3E1D1E013C0052710E000C0000075
:100580000BB91AC0052710E0221F1DC010E021C0C2
:100590004AE502C032ED432FC4E1D0E032E01AB1A7
:1005A0001660599A0BB11AB956E020E865E320FFAE
:1005B00005270BB9279517951C3FF0F66695B8F7F8
:1005C000B1F720FF05270BB9279517951C3FD0F6EB
:1005D0002795179517FF052700001C3F0BB9B0F6AC
:1005E00029913A9519F7097F10912401110FC651ED
:1005F000D0400BB911F010931E0111E01CBB02603A
:100600001AB1197F402F497F54E05A95F1F70BB981
:100610001AB94BB97FCFDC0113963C911397F32F96
:1006200014962C911497E22F12969C911297903366
:1006300039F42370E22FF0E0EE5FFE4F80810895E1
:10064000983529F431110EC0E1E0F0E006C0903594
:1006500099F431110CC0E0E0F0E089E0809357009C
:1006600084910895383091F5E3E0F0E0F6CF38302A
:1006700069F5E2E0F0E0F1CF903241F4CF01A0E083
:10068000B0E0880F991FAA1FBB1F0CC0983271F4ED
:10069000CF01A0E0B0E0880F991FAA1FBB1F0196F1
:1006A000A11DB11DABBFFC0187910895903A11F4D3
:1006B000CF0189C2903C29F415966C91CF0190D25C
:1006C00005C09F3F19F481EF8093110180E00895E8
:1006D0001AB881E08BB985BF92E095BFE0E0F1E701
:1006E000A89531979040E1F704B603FE0EC08EEF57
:1006F0009FE071D2C1E0803B904B09F0C0E06FEF0A
:100700007FEF8EEF9FE07AD208C004B601FE04C0EE
:10071000C9B1C170C82701C0C0E014BEC1110CC06E
:10072000F894519A1BB81DBA1092690081E085BFF8
:1007300015BEE0E0F0E009958EEF8093110114BE44
:100740000FB6F894A895809160008861809360004E
:10075000109260000FBE80916900826080936900F2
:10076000E89A519A8CE0E0E0F5E3A8953197804053
:10077000E1F75198789481EF809311011091230152
:10078000135017FD74C180912001CCE0D0E0C81B4C
:10079000D109C95DDE4F80911F018D3209F0C0C0C3
:1007A000183009F062C183EC809313018AE58093CD
:1007B0000101109212013881832F8076998188235C
:1007C00009F43FC046E051E05093220140932101DB
:1007D000933031F4CE011FDF8093090184E096C08D
:1007E000953009F492C09A3009F48FC08CEF890FCC
:1007F0008630E0F44A815B8150930E0140930D01F5
:10080000993039F48C819D819093100180930F0170
:1008100014C08E8180930C012D81227020930B01D6
:1008200090930A0137FD6DC08FEF6BC0809111016D
:10083000923029F48E7F8093110180E067C081603F
:10084000FACF8A8110921C01911106C010921D01ED
:100850002CE131E082E050C0953019F480932401FE
:100860003DC09630A9F59B81913019F48EEB90EE46
:1008700004C0923041F48CEA90EE90932201809370
:10088000210182E121C09330F1F4811108C08AEF87
:1008900090EE909322018093210184E015C0813075
:1008A00041F48EED90EE90932201809321018CE132
:1008B0000BC0823041F480ED90EE90932201809342
:1008C00021018EE001C080E090E4909312011EC0EF
:1008D000983079F0993031F4809326012CE131E0A1
:1008E00080E00AC081E09A3009F080E02CE131E03C
:1008F00003C026E231E081E0309322012093210100
:1009000005C090E89093120108C081E09F81911189
:1009100004C09E81981708F4892F80930001A5C018
:100920008091120187FFA1C000910C01011708F40A
:10093000102F011B00930C01F12CF11608F091C04F
:1009400080910A018730A0F06E01FFEFCF1ADF0A15
:10095000688180910D0190910E019C012F5F3F4FA6
:1009600030930E0120930D013BD1F394E601E5CFC6
:1009700080910D0190910E01A0910F01B091100195
:100980008115904EA140B10508F06DC0F394F39429
:10099000F89440910D0150910E0160910F017091FA
:1009A00010012991399181E00901FA0160935B00FE
:1009B00080935700E8951124789480910D019091CF
:1009C0000E01A0910F01B09110010296A11DB11D61
:1009D00080930D0190930E01A0930F01B09310012D
:1009E000882351F00111A9CFF11608F4A6CF809108
:1009F0000B01882309F4A1CFF89480910D01909107
:100A00000E01A0910F01B09110010297A109B10947
:100A100023E0FC01A0935B0020935700E8957894B5
:100A200007B600FCFDCFF89480910D0190910E0166
:100A3000A0910F01B09110010297A109B10925E021
:100A4000FC01A0935B0020935700E895789407B6CB
:100A500000FCFDCFF89481E180935700E8957894ED
:100A60006CCF011102C010920001109223018091FD
:100A7000010184FF7EC0809100018F3F09F479C09D
:100A8000C82F893008F0C8E08C1B8093000190913A
:100A9000130188E8892780931301CC2309F48DC0C2
:100AA0008091120187FF37C080910C018C1708F4E8
:100AB000C82F8C1B80930C01B0900A01D0E004E198
:100AC00011E0CD1709F449C0C0900D01D0900E017E
:100AD000E0900F01F090100186E08B1530F48091CA
:100AE0000D0190910E016FD003C0EBBEF60187910E
:100AF000F80180830F5F1F4FFFEFCF1ADF0AEF0A65
:100B0000FF0AC0920D01D0920E01E0920F01F09207
:100B10001001DF5FD6CFA0912101B091220186FFA5
:100B200011C024E131E08C2FAD0160E070E0616024
:100B30006BBFFA014791F90141939F0111968150D2
:100B400099F707C0E4E1F1E08C2F9D9191938150DA
:100B5000E1F7B0932201A09321016C2F84E191E091
:100B600042DCCC5FCC3019F08FEF80930001C09352
:100B7000010184E199B1967031F48150D9F7109256
:100B8000240110921E0180911101803130F0489BA8
:100B90000FC080911101805109C0489909C080910E
:100BA0001101823028F0809111018250809311014F
:100BB000809111018111E2CDB3CD60E084E191E03B
:100BC00012DCC4E0D1CFF999FECF92BD81BDF89A75
:100BD000992780B50895A8E1B0E042E050E013C045
:100BE000262FF999FECF1FBA92BD81BD20BD0FB649
:100BF000F894FA9AF99A0FBE01960895F1DF272F1B
:100C0000F0CFDC01CB01FC01F999FECF06C0F2BDAB
:100C1000E1BDF89A319600B40D9241505040B8F7BA
:100C20000895F894FFCFFF5A1E9705008F929F9268
:100C3000AF92BF92CF92DF92EF92FF920F931F93EA
:100C4000CF93DF93CDB7DEB7DA950FB6F894DEBF5A
:100C50000FBECDBF14BE0FB6F894A895809160006A
:100C6000886180936000109260000FBEF894198232
:100C7000209100013091010180E090EEA1E0B0E010
:100C8000A901032E000C660B770B6BBFFA0147918D
:100C90005691ABBFFC01679176914617570719F043
:100CA00081E089830CC02E5F3F4F0296A11DB11DCC
:100CB000823C49EE940741E0A407B10509F7898118
:100CC000882309F491C02CE8C22E20EED22EEE2407
:100CD000E394F12CB701A601442720E031E0CE01D6
:100CE000019618DAC701B6016C58744E8F4F9F4FAA
:100CF0000CE510E020E031E0AE014F5F5F4F30DAED
:100D00008FEFD81AE80AF80A4CE8C41644EED40665
:100D100041E0E406F104F1F6812C90EE992EAA242C
:100D2000A394B12CE12CF12C40E051E06FEF70E086
:100D3000CE0101966ED040910001509101014E0DFF
:100D40005F1D052E000C660B770B20E031E0CE0115
:100D50000196E0D903E710E020E031E0AE014F5FFB
:100D60005F4FC501B401FCD98FEF981AA80AB80AE1
:100D7000E11445E0F40611F0F394D6CF82ECC82ECE
:100D800084E0D82E40E051E06FEF70E0CE01019694
:100D900040D0960141E0C416D40610F020E031E0C6
:100DA00040910001509101014E0D5F1D052E000C78
:100DB000660B770BCE010196ADD9C701A0E0B0E07C
:100DC000BC01CD0170528E4F9F4F0CE510E020E02A
:100DD00031E0AE014F5F5F4FC3D9F394DA9482ECF8
:100DE000E81689E0F80670F280E090E0D3950FB63F
:100DF000F894DEBF0FBECDBFDF91CF911F910F9151
:100E0000FF90EF90DF90CF90BF90AF909F908F902A
:100E10000895DC0101C06D9341505040E0F7089502
:040E2000F894FFCF74
:020E24006A0260
:00000001FF
